:100000000C9480050C94E1050C94E1050C94D30646
:100010000C94E1050C94E1050C94E1050C94E105C8
:100020000C94E1050C94E1050C94E1050C94E80FA7
:100030000C9497100C94CE1D0C94E1050C94E105E2
:100040000C94E1050C94E1050C94E1050C94421E1E
:100050000C94E1050C94E1050C94E1050C94E10588
:100060000C94E1050C94E1050C94E1050C94E10578
:100070000C94E1054E0E750E6D0F750E6D0FC10ED1
:10008000E40E6D0F3B0F4A0FDF13DF130914091441
:1000900064149814A616A616AF14A6169A159A15E7
:1000A0006016A6167516931680680169023A3B43DE
:1000B0003C443D453E7E3F734041427A524846476C
:1000C000506A6B514F291E1F2021222324252627E9
:1000D0002D2E352A490354557C6C636D4A2B141A16
:1000E0000815171C180C12132F304C655F606156F1
:1000F0006E6F4D8078041607090A0B0D0E0F33340E
:100100003128585C5D5E62704B7153791D1B061976
:100110000511103637387D75595A5B77760072397C
:100120007B2C7F4E64578080253032580A007265E0
:10013000736574206661696C3A2000253032580A74
:10014000006C61796F75743A2000253032580A00CE
:1001500072657365743A2000200025303258002003
:10016000446F6E650A002E005265736574696E6790
:1001700020004C45443A20253032580A00556E6B19
:100180006E6F776E20657874726120636F6D6D613C
:100190006E643A20253032580A006C61796F7574AC
:1001A0000A004C454420616C6C206F66660A004C66
:1001B000454420616C6C206F6E0A00436C69636B70
:1001C000204F66660A00436C69636B204F6E0A001D
:1001D00042656C6C204F66660A0042656C6C204F6D
:1001E0006E0A0052657365740A0044656C65746537
:1001F0003A20202020202052657365740A00496E41
:10020000736572743A2020202020204C61796F752C
:10021000740A005067446F776E3A20202020202017
:100220004C454420616C6C204F66660A005067554F
:10023000703A20202020202020204C454420616C52
:100240006C204F6E0A00456E643A2020202020204A
:10025000202020546F67676C6520436C69636B0ACC
:1002600000486F6D653A2020202020202020546F08
:1002700067676C652042656C6C0A000A0A2D2D2D9B
:100280002D2D2053756E20636F6E766572746572C6
:100290002048656C70202D2D2D2D2D0A000A4B65F0
:1002A00079626F6172642073746172742E0A000A3D
:1002B00055534220636F6E666967757265642E0AD6
:1002C000000A0A544D4B3A65363361666638372F5B
:1002D0004C5546410A0A002E03530075006E00205B
:1002E000006B006500790062006F006100720064BD
:1002F00000200063006F006E0076006500720074DD
:10030000006500720000000E0374002E006D002EC8
:10031000006B002E000000040309040902740004AD
:100320000100A032090400000103010100092111AC
:100330000100012240000705810308000A090401A9
:10034000000103010200092111010001224D0007F3
:1003500005820308000A09040200010300000009E5
:1003600021110100012236000705830308000A0954
:1003700004030002030000000921110100012222F0
:100380000007058403200001070504032000011273
:1003900001100100000008EDFE33330001010200EE
:1003A000010631FF0974A1010975150026FF0095AA
:1003B00020750881020976150026FF009520750832
:1003C0009102C005010980A10185021601002637AE
:1003D000001A81002AB700751095018100C0050C34
:1003E0000901A1018503160100269C021A01002AB9
:1003F0009C02751095018100C005010902A1010947
:1004000001A10005091901290515002501950575AA
:10041000018102950175038101050109300931153A
:1004200081257F95027508810609381581257F95FC
:100430000175088106050C0A38021581257F950192
:1004400075088106C0C005010906A101050719E06C
:1004500029E71500250195087501810295017508A8
:10046000810105081901290595057501910295017C
:10047000750391010507190029FF150026FF009556
:100480000675088100C0636F6E73756D65723A20E2
:10049000253034580A0073797374656D3A2025301D
:1004A00034580A000A002530325820006B65796202
:1004B0006F6172643A20004C45443A20253032582E
:1004C0000A00253032583A202530386225730A0058
:1004D000722F632030313233343536370A00290A1F
:1004E000002575002F002575005D2800256400207B
:1004F00000256400200025640020002564007C00A5
:1005000025303258006D6F7573656B6579205B62BD
:10051000746E7C782079207620685D287265702F53
:1005200061636C293A205B006D6B5F776865656C71
:100530005F74696D655F746F5F6D6178203D202524
:10054000640A006D6B5F776865656C5F6D61785FED
:100550007370656564203D2025640A006D6B5F74CF
:10056000696D655F746F5F6D6178203D2025640A59
:10057000006D6B5F6D61785F7370656564203D2011
:1005800025640A006D6B5F696E74657276616C201C
:100590003D2025640A006D6B5F64656C6179203DC8
:1005A0002025640A006D6B5F776865656C5F746910
:1005B0006D655F746F5F6D6178203D2025640A0072
:1005C0006D6B5F776865656C5F6D61785F73706593
:1005D0006564203D2025640A006D6B5F74696D655C
:1005E0005F746F5F6D6178203D2025640A006D6B3C
:1005F0005F6D61785F7370656564203D2025640AD6
:10060000006D6B5F696E74657276616C203D2025AC
:10061000640A006D6B5F64656C6179203D20256420
:100620000A000A00257500363A20776865656C5F18
:1006300074696D655F746F5F6D61783A20000A00C0
:10064000257500353A20776865656C5F6D61785F68
:1006500073706565643A20000A00257500343A20FD
:1006600074696D655F746F5F6D61783A20000A0090
:10067000257500333A206D61785F73706565643A63
:1006800020000A00257500323A20696E7465727682
:10069000616C286D73293A20000A00257500313AF3
:1006A0002064656C6179282A31306D73293A200005
:1006B0000A092D2056616C756573202D0A004D3E88
:1006C000004D25643E20003F00736574206465661C
:1006D00061756C740A00433E20007768657265207E
:1006E00064656C74613A20637572736F723D256442
:1006F0002C20776865656C3D25640A536565206824
:100700007474703A2F2F656E2E77696B697065640B
:1007100069612E6F72672F77696B692F4D6F7573E3
:10072000655F6B6579730A000A092D204D6F75733B
:10073000656B6579202D0A4553432F713A09717510
:1007400069740A313A0964656C6179282A31306D1F
:1007500073290A323A09696E74657276616C286D84
:1007600073290A333A096D61785F73706565640AAD
:10077000343A0974696D655F746F5F6D61780A352D
:100780003A09776865656C5F6D61785F7370656560
:10079000640A363A09776865656C5F74696D655FF0
:1007A000746F5F6D61780A0A703A097072696E74CD
:1007B0002076616C7565730A643A09736574206408
:1007C000656661756C74730A75703A092B310A6439
:1007D0006F776E3A092D310A706775703A092B31BF
:1007E000300A7067646F776E3A092D31300A0A73E8
:1007F00070656564203D2064656C7461202A206DFD
:1008000061785F7370656564202A20287265706561
:100810006174202F2074696D655F746F5F6D6178FE
:10082000290A003F004D3E2000433E20004C256435
:100830000A000A092D20436F6E736F6C65202D0A24
:100840004553432F713A09717569740A6D3A096D00
:100850006F7573656B65790A000A092D204D616714
:100860006963202D0A643A0964656275670A783AFB
:10087000096465627567206D61747269780A6B3A04
:10088000096465627567206B6579626F6172640ADD
:100890006D3A096465627567206D6F7573650A76D8
:1008A0003A0976657273696F6E0A733A09737461F7
:1008B0007475730A633A09636F6E736F6C65206DAC
:1008C0006F64650A302D343A096C61796572302D98
:1008D00034284631302D4634290A506175733A095F
:1008E000626F6F746C6F616465720A003F007469B7
:1008F0006D65725F72656164333228293A20253054
:10090000346C580A006B6579626F6172645F696468
:100910006C653A2025580A006B6579626F617264D4
:100920005F70726F746F636F6C3A2025580A0068AD
:100930006F73745F6B6579626F6172645F6C65641D
:100940007328293A2025580A000A092D205374617A
:10095000747573202D0A004743433A20352E342EF8
:1009600030204156522D4C4942433A20322E302EEF
:1009700030204156525F415243483A2061767233EB
:10098000350A004F5054494F4E533A204C5546417A
:10099000204D4F5553454B45592045585452414BD6
:1009A000455920434F4E534F4C4520434F4D4D41E9
:1009B0004E44204B45594D41505F53454354494F98
:1009C0004E20424F4F544C4F414445525F53495A79
:1009D000450A004255494C443A2065363361666603
:1009E0003837202831333A35363A35352041707260
:1009F0002020392032303230290A005649443A202A
:100A000030784645454428742E6D2E6B2E29205093
:100A100049443A203078333333332853756E206B92
:100A20006579626F61726420636F6E76657274655A
:100A30007229205645523A203078303130300A0041
:100A4000444553433A20636F6E7665727473205346
:100A5000756E206B6579626F6172642070726F745D
:100A60006F636F6C20696E746F205553420A000AE1
:100A7000092D2056657273696F6E202D0A000A6D6C
:100A80006F7573653A206F66660A000A6D6F75733D
:100A9000653A206F6E0A000A6B6579626F61726455
:100AA0003A206F66660A000A6B6579626F6172644C
:100AB0003A206F6E0A000A6D61747269783A206F8D
:100AC00066660A000A6D61747269783A206F6E0A70
:100AD000000A64656275673A206F6E0A000A6465F1
:100AE0006275673A206F66660A000A0A626F6F7461
:100AF0006C6F616465722E2E2E2000433E20000034
:100B000011241FBECFEFD4E0DEBFCDBF04B603FE7D
:100B100041C080916A0390916B03A0916C03B091E6
:100B20006D038730904BA740B04BA1F510926A033C
:100B300010926B0310926C0310926D0314BE0FB6EB
:100B4000F894A8958091600088618093600010926D
:100B500060000FBE1092010810920008E3E0F0E080
:100B600089E080935700E491E695E370E150E3302B
:100B700040F4F0E0EE0FFF1FE25DFE4F80819181B7
:100B800002C080E090E1E0E0F0E8E81BF90BF695A8
:100B9000E795099511E0A0E0B1E0E2E9FDE402C0CB
:100BA00005900D92AE33B107D9F723E0AEE3B1E083
:100BB00001C01D92AA36B207E1F70E94760B0C9491
:100BC000C7260C940000FF93EF93E0913E01F09153
:100BD0003F01309709F00995EF91FF910895FC01CD
:100BE0008591803011F0EFDFFBCF0895FF27E0E221
:100BF00030E247FF0CC0419597FF09C0EDE26095D8
:100C0000709580959095611D711D811D911D27FF27
:100C100002C0219530E350E2AA27660F771F881F94
:100C2000991FAA1FA41710F0A41B63955A95A9F742
:100C3000AA3008F0A95FA05DAF93F3956115710527
:100C40008105910541F7ED3211F4EF93F395F21719
:100C500018F43F93F395FBCF8F91B5DFFA95E1F749
:100C60000895E991F9918591803021F0853219F04C
:100C7000AADFF9CF089520E0E89455915532C1F3E9
:100C8000503311F4689455915A3348F4505390F30B
:100C9000220F022E220F220F200D250FF4CF0EF46B
:100CA000219589919991533619F3533729F1533589
:100CB00059F1BC0188279927E8945C3621F4899181
:100CC000999168945591543639F446EF7EF077FF48
:100CD0000DC08FEF9FEF0AC055374AE039F0583505
:100CE00040E121F0523642E009F00895FF93EF937E
:100CF0007DDFEF91FF91B7CFFF93EF93FC018191DF
:100D00008030B9F360DFFBCFFF93EF9368DFF1CF63
:100D1000DF93CF93CDB7DEB72596A3DFCF91DF91D9
:100D2000089552985A9AE9E6F0E0808180638083C2
:100D3000EA9A7894539A5B980895209140018091A3
:100D40004101821761F030E0F901EE5BFE4F8081D6
:100D50002F5F3F4F2770332720934001089580E095
:100D600008955B9AE3E0FDE03197F1F700C00000E1
:100D700028E030E091E0482F492311F05B9801C052
:100D80005B9AE3E0FDE03197F1F700C00000990FB6
:100D90002150310981F75B9883E09DE00197F1F7DD
:100DA00000C0000008951F920F920FB60F921124F9
:100DB0002F933F934F935F938F939F93EF93FF9363
:100DC0008FE796E00197F1F700C0000088E090E01F
:100DD00021E040E0E3E0FDE03197F1F700C00000E2
:100DE0004A9B422B220F0197A9F783E09DE00197D0
:100DF000F1F700C000008091410190E09C012F5F5D
:100E00003F4F2770332750914001521731F0FC01BA
:100E1000EE5BFE4F40832093410184E08CBBFF9149
:100E2000EF919F918F915F914F913F912F910F90F3
:100E30000FBE0F901F901895569A5E9A0E949106C9
:100E4000EAE4F1E0119221E0EA35F207D9F788E609
:100E500091E00E94EF0586E691E00E94EF050E9476
:100E60009D068111FCCF81E00E94B1068FEF99E6CB
:100E700028E1815090402040E1F700C000000E942E
:100E80009D068F3F41F78FEF99E628E18150904012
:100E90002040E1F700C000000E949D068430D9F692
:100EA0008FE591E00E94EF055E9808951F93CF9320
:100EB000DF930E949D06C82F882309F476C0809195
:100EC0004C0380FF0CC01F92CF938AE591E09F9363
:100ED0008F930E9488060F900F900F900F90809133
:100EE0004C0380FF04C088E591E00E94EF05CF37F6
:100EF00009F45DC0B8F4CE3709F061C08EE291E02C
:100F00000E94EF052FEF89E698E121508040904044
:100F1000E1F700C000000E949D061F928F9388E2B7
:100F200091E03BC0CE3F31F1CF3F09F048C080E5B2
:100F300091E00E94EF052FEF89E698E12150804073
:100F40009040E1F700C000000E949D06C82F1F924C
:100F50008F938AE491E09F938F930E9488060F906D
:100F60000F900F900F90C43001F50E94E1100E9485
:100F70001A081BC081E491E00E94EF052FEF89E67B
:100F800098E1215080409040E1F700C000000E94AD
:100F90009D061F928F938BE391E09F938F930E9406
:100FA00088060F900F900F900F9080E039C0EAE410
:100FB000F1E0119221E0EA35F207D9F7F6CF1C2FC4
:100FC0001770DC2FD695D695D695C7FF15C0DF7064
:100FD000612F8D2F0E944812882309F1ED2FF0E038
:100FE000E65BFE4F81E090E001C0880F1A95EAF7BA
:100FF00080959081892312C0612F8D2F0E94481205
:1010000081110DC0ED2FF0E0E65BFE4F81E090E036
:1010100001C0880F1A95EAF79081892B80838C2F65
:10102000DF91CF911F910895E82FF0E0E65BFE4F2E
:1010300080810895CF93C82FC17083FDC26082FD67
:10104000C46081FDC8601F928F9382E791E09F93F7
:101050008F930E9488068EE00E94B1060F900F9039
:101060000F900F908C2FCF910C94B106CF938A34B0
:1010700009F440C048F48833D1F0893409F46DC0D4
:101080008B3009F073C013C08C3471F108F45CC06C
:101090008D3409F443C08E3409F068C082EA91E0CF
:1010A0000E94EF058EE00E94B10680E05BC08BE7F6
:1010B00092E00E94EF0581E692E00E94EF0586E44F
:1010C00092E00E94EF058DE292E00E94EF0583E13D
:1010D00092E00E94EF058EEF91E00E94EF058AEE0C
:1010E00091E00E94EF054EC083EE91E00E94EF0573
:1010F00081E038C0C0915B0181E0C827C0935B01EB
:10110000CC2331F08AED91E00E94EF0582E013C01C
:1011100080ED91E00E94EF0583E024C0C0915A0168
:1011200081E0C827C0935A01CC2341F086EC91E0BE
:101130000E94EF058AE00E94B10625C08BEB91E08A
:101140000E94EF058BE00EC08FEA91E00E94EF0550
:101150008EE00E94B1068FEF05C08AE991E00E94FF
:10116000EF058FE00E94B106C1E00DC01F928F9382
:101170008DE791E09F938F930E9488060F900F90C8
:101180000F900F90C0E08C2FCF910895809168024E
:101190000895CF93DF9300D01F92CDB7DEB79C01A7
:1011A00080916103843019F593E099833B832A830E
:1011B0009093E9008FEF9091E800815095FD06C073
:1011C00095ED9A95F1F700008111F5CF8091E80037
:1011D00085FF0DC040E050E063E070E0CE01019675
:1011E0000E94210D8091E8008E778093E8000F9097
:1011F0000F900F90DF91CF910895CF93DF9300D0A0
:101200001F92CDB7DEB720916103243031F522E083
:101210002983805891099B838A8383E08093E90026
:101220008FEF9091E800815095FD06C095ED9A955D
:10123000F1F700008111F5CF8091E80085FF0DC026
:1012400040E050E063E070E0CE0101960E94210D85
:101250008091E8008E778093E8000F900F900F90B8
:10126000DF91CF910895209161032430F1F422E0C1
:101270002093E9002FEF3091E800215035FD06C0A2
:1012800035ED3A95F1F700002111F5CF2091E800F6
:1012900025FF0BC040E050E065E070E00E94210DAA
:1012A0008091E8008E778093E8000895CF93DF93D4
:1012B00020916103243049F521E02093E90021E8E1
:1012C000215059F03091E80035FD07C0EFE3F1E01F
:1012D0003197F1F700C00000F3CF2091E80025FF1F
:1012E00014C0EC0140E050E068E070E00E94210D85
:1012F0008091E8008E778093E80088E0FE01A0E608
:10130000B2E001900D928A95E1F7DF91CF910895B7
:10131000CF93C0915E01C1110BC00E940C1E643CB2
:1013200079408105910520F081E080935E01C1E064
:101330008C2FCF910895FF920F931F93CF93DF933C
:10134000D82F0FB607FE83C080916103843081F0EF
:101350008091030190E001962091050130E0822305
:1013600093232091040130E08217930709F0C9C04C
:101370000E948809811110C08091030190E00196BC
:101380002091050130E0822393232091040130E075
:101390008217930709F0B5C00E94001E8C01C0910E
:1013A000E900CF709091EC00892F817090FD80E86A
:1013B000C82B84E08093E90085E0F82E8091EB0053
:1013C00085FD42C08091EB0080FF3EC08091EE0021
:1013D00087FF3AC08091040190910301981709F4A6
:1013E00057C09091E80095FF8AC0E0910101F0910B
:1013F0000201E80FF11D20818F5F90910501892383
:10140000809304012093F1008091E80085FDE2CFF4
:101410008091E80080FFDECF8091E8008E77809396
:10142000E800F0920001D6CF8091030190E0019690
:101430002091050130E0822393232091040130E0C4
:101440008217930709F448C0CF70C093E900409118
:101450000301842F90E001962091050130E0822362
:1014600093232091040130E08217930709F44CC0C4
:10147000E0910101F0910201E40FF11DD083809110
:1014800003018F5F909105018923809303013CC084
:101490008091E80085FF33C0D093F10081E0909106
:1014A000F200992391F09091E80090FF0EC0909186
:1014B000E80095FF03C01092F100F9CF9091E80089
:1014C0009E779093E800F0920001882309F4ACCF56
:1014D000CF70C093E90018C080910001882309F4FF
:1014E000B3CF0E94001E9C018017910711F489015F
:1014F00065CF90910001915090930001F8CF80E06A
:10150000CECF40910301B4CF80E0DF91CF911F9106
:101510000F91FF900895089542E061EC81E00E94F0
:101520009A0C42E061EC82E00E949A0C42E061EC8D
:1015300083E00E949A0C42E261EC84E00C949A0CE5
:1015400080916303833009F453C030F4813071F02B
:10155000823009F48CC008958A3009F478C08B3049
:1015600009F45EC0893009F09AC020C080916203FE
:10157000813A09F094C08091E800877F8093E80069
:101580008091660390916703892B21F468E080E6DF
:1015900092E003C060E080E090E070E00E946C0D9B
:1015A0008091E8008B778093E80008958091620332
:1015B000813209F074C08091660390916703892B92
:1015C00009F06DC08091E800877F8093E8008091EA
:1015D000E80082FD05C0809161038111F8CF5FC0F2
:1015E0008091F100809368028091E8008B7753C06E
:1015F00080916203813A09F052C080916603909114
:101600006703892B09F04BC08091E800877F8093A6
:10161000E8008091E80080FFFCCF8091100136C087
:10162000809162038132D9F58091660390916703BE
:10163000892BA9F58091E800877F8093E8000E94BC
:10164000CF0C80916403809310010C948F138091D0
:101650006203813221F58091E800877F8093E80062
:101660000E94CF0C80916503809369020895809158
:101670006203813AA1F48091E800877F8093E800BB
:101680008091E80080FFFCCF809169028093F10097
:101690008091E8008E778093E8000C94CF0C089539
:1016A0008091680280935F01109268020E94461246
:1016B0000C948F130C94500B0E948D1D80915F032E
:1016C000882329F00E94B61D81110C94840C089582
:1016D0000E94CA1D80915F018093680208950C9456
:1016E000680B08950C94710B0C94710BCF9384B715
:1016F000877F84BF0FB6F894A895809160008861B9
:1017000080936000109260000FBE90E080E80FB6FA
:10171000F89480936100909361000FBE8BE999E08B
:101720000E94601D86E091E00E94DC1081EC92E056
:101730000E94EF050E94740B0E949B110E94850F6E
:101740000E94D80F78940E949D118091610384308B
:1017500019F00E94710BF9CF8FEA92E00E94EF0519
:101760000E94720B8DE992E00E94EF05C4E0809127
:101770006103853019F40E945C0BF9CF0E94A1111E
:101780002091E4003091E50080915C0190915D0131
:101790002817390761F38091E4009091E500909358
:1017A0005D0180935C010E948809882301F3809188
:1017B00061038430E1F68091E9008F702091EC00A4
:1017C000922F917020FD90E8892BC093E9009091B1
:1017D000EB0090FF3FC09091EE0097FF3BC09091CF
:1017E000040120910301291709F12091E80025FF48
:1017F0001DC0E0910101F0910201E90FF11D30815E
:101800009F5F209105019223909304013093F10092
:101810009091E80095FDE3CF9091E80090FFDFCF35
:101820009091E8009E779093E800D9CF9091F200D4
:10183000992381F09091E80090FF0CC09091E8000E
:1018400095FF03C01092F100F9CF9091E8009E77C8
:101850009093E8008F708093E90089CF292F332778
:1018600023303105C9F060F42130310581F0223098
:10187000310509F041C084E790E02BE133E040C03E
:1018800021323105E1F02232310531F135C082E1FA
:1018900090E02FE833E034C099278130910549F07A
:1018A00028F0029749F5E7EDF2E005C0E7E1F3E043
:1018B00002C0E7E0F3E0849190E09F0121C0643032
:1018C0007105D0F4660F771FFB01EB5DFE4F2081A1
:1018D000318189E090E014C06430710568F4FB0147
:1018E000EE0FFF1FE35EFE4F20813181FB01E75EBB
:1018F000FE4F808190E004C080E090E020E030E086
:10190000FA0131832083089584E089BD86E089BD92
:1019100009B400FEFDCF8091D8008F7D8093D80060
:101920008091E00082608093E0008091E00081FD82
:10193000FCCF0895982F953068F59093E90098179B
:1019400039F07091EC002091ED005091F00003C04F
:10195000242F762F50E021FD02C09F5FECCF309105
:10196000EB003E7F3093EB003091ED003D7F3093F4
:10197000ED003091EB0031603093EB007093EC00A0
:101980002093ED005093F0002091EE0027FDE5CF6D
:1019900080E008958F708093E90081E00895809140
:1019A000620387FF11C08091E80082FD05C080912D
:1019B00061038111F8CF11C08091E8008B770BC0D3
:1019C00080916103882349F08091E80080FFF8CF7F
:1019D0008091E8008E778093E80008952091E400DC
:1019E0003091E50095E64091EC00842F817040FF36
:1019F00023C08091E80080FD1DC080916103882391
:101A000099F0853099F08091EB0085FD11C04091EF
:101A1000E4005091E5002417350729F3915011F0A7
:101A20009A01E1CF84E0089582E0089583E008956B
:101A300081E0089580E008954091E80042FFDDCF05
:101A40000895CF92DF92EF92FF920F931F93CF935F
:101A5000DF93EC018B017A010E94EE0C811133C0FF
:101A6000E114F10439F0F70180819181081B190B11
:101A7000C80FD91FC12CD12C0115110519F1809166
:101A8000E80085FD16C08091E8008E778093E8001D
:101A9000E114F10449F0F70180819181C80ED91E4B
:101AA000D182C08285E00FC00E94EE0C882321F312
:101AB0000AC089918093F10001501109FFEFCF1AFC
:101AC000DF0ADACF80E0DF91CF911F910F91FF9075
:101AD000EF90DF90CF9008952091680330916903D3
:101AE0002617370748F06115710539F42091E80091
:101AF0002E772093E80001C0B901FC0120E06115B8
:101B0000710561F1809161038823D9F18530D9F1A4
:101B10008091E80083FD39C08091E80082FD2BC0F0
:101B20008091E80080FFEBCF8091F20090E061159A
:101B3000710551F08830910538F421912093F1001E
:101B4000615071090196F3CF21E0089709F020E078
:101B50008091E8008E778093E800D1CF2111D2CF19
:101B60000AC080916103882361F0853061F0809123
:101B7000E80083FD0AC08091E80082FFF2CF80E098
:101B8000089582E0089583E0089581E0089520910A
:101B90006803309169032617370748F0611571050E
:101BA00039F42091E8002E772093E80001C0B901B4
:101BB000FC0120E06115710579F1809161038823B2
:101BC00009F43DC0853009F43CC08091E80083FDF4
:101BD0003AC08091E80082FD2CC08091E80080FF2F
:101BE000E9CF8091F20090E06115710559F08830DD
:101BF000910540F424912093F100319661507109D0
:101C00000196F2CF21E0089709F020E08091E800EA
:101C10008E778093E800CECF2111CFCF0AC080917C
:101C20006103882361F0853061F08091E80083FDD5
:101C30000AC08091E80082FFF2CF80E0089582E040
:101C4000089583E0089581E008951F93CF93DF9373
:101C5000CDB7DEB7AA970FB6F894DEBF0FBECDBFE3
:101C6000E2E6F3E08091F100819323E0EA36F207A7
:101C7000C9F70E94A00A8091E80083FF2EC18091DD
:101C8000620390916303492F50E04A30510508F0F8
:101C900024C1FA01E65CFF4F0C94AD26803821F098
:101CA000823809F01AC108C080915E0390915F03E9
:101CB000992389F082600FC0809166038F70853010
:101CC00008F00BC18093E9008091EB0085FB882729
:101CD00080F91092E9009091E800977F9093E800D6
:101CE0008093F1001092F100D1C0282F2D7F09F0D0
:101CF000F4C0882319F0823061F0EFC08091640352
:101D0000813009F0EAC0933009F080E080935F03EE
:101D10002EC08091640381112AC0809166038F7068
:101D20002FEF280F243008F0D8C08093E9002091CD
:101D3000EB0020FF1CC0933021F48091EB00806207
:101D400014C09091EB0090619093EB0021E030E0A3
:101D5000A90102C0440F551F8A95E2F74093EA009B
:101D60001092EA008091EB0088608093EB00109263
:101D7000E9008091E800877F8093E8000E94CF0C03
:101D8000ACC08111AAC0109164031F778091E30059
:101D90008078812B8093E3008091E800877F809397
:101DA000E8000E94CF0C8091E80080FFFCCF80917A
:101DB000E30080688093E300111102C082E001C05B
:101DC00083E08093610389C08058823008F085C029
:101DD00080916403909165038C3D53E0950779F5FC
:101DE00083E08A838AE289834FB7F894DE011396F1
:101DF00020E03EE051E2E32FF0E050935700E49101
:101E000020FF03C0E295EF703F5FEF708E2F90E0F0
:101E1000EA3010F0C79601C0C0968D939D932F5F56
:101E2000243149F74FBF8091E800877F8093E80015
:101E30006AE270E0CE0101960E946C0D16C06091BE
:101E4000660370916703AE014F5F5F4F0E942E0CD7
:101E5000BC01892B09F441C09091E800977F9093D1
:101E6000E80089819A810E94C70D8091E8008B77F4
:101E70008093E80032C0803881F58091E800877F48
:101E80008093E80080915D038093F1008091E800E9
:101E90008E7772CF811121C0809164039091650388
:101EA00099270297D4F48091E800877F8093E80017
:101EB0008091640380935D030E94CF0C80915D0349
:101EC000811106C08091E30087FD02C081E001C05E
:101ED00084E0809361030E948C0A8091E80083FF74
:101EE0000AC08091E800877F8093E8008091EB0032
:101EF00080628093EB00AA960FB6F894DEBF0FBE07
:101F0000CDBFDF91CF911F9108950E94E20F0E94F3
:101F1000E50FE0EEF0E0808181608083E8EDF0E0A5
:101F200080818F77808319BCE3E6F0E08081816057
:101F300080831092600308950E94E20F0E94E50FD3
:101F40008091D8008F778093D8008091D8008068E6
:101F50008093D8008091D8008F7D8093D80084E052
:101F600089BD86E089BD09B400FEFDCF10926103F2
:101F700010925D0310925F0310925E0342E060E0F6
:101F800080E00E949A0C8091E1008E7F8093E100B6
:101F90008091E20081608093E2008091E20088609D
:101FA0008093E2008091E0008E7F8093E0000895AE
:101FB000E3E6F0E080818E7F808381E080936003A0
:101FC0000C949C0F1092E20008951092E100089585
:101FD0001F920F920FB60F9211242F933F934F939E
:101FE0005F936F937F938F939F93AF93BF93EF9381
:101FF000FF938091E10082FF0BC08091E20082FF9D
:1020000007C08091E1008B7F8093E1000E94DB108C
:102010008091E10080FF19C08091E20080FF15C02F
:102020008091E2008E7F8093E2008091E2008061E7
:102030008093E2008091D80080628093D80019BC20
:1020400085E0809361030E945A0B8091E10084FF38
:1020500030C08091E20084FF2CC084E089BD86E01E
:1020600089BD09B400FEFDCF8091D8008F7D80939B
:10207000D8008091E1008F7E8093E1008091E200A2
:102080008F7E8093E2008091E20081608093E20085
:1020900080915D03882311F084E007C08091E30004
:1020A00087FD02C081E001C083E0809361030E944C
:1020B0006F0B8091E10083FF29C08091E20083FFD4
:1020C00025C08091E100877F8093E10082E08093CA
:1020D000610310925D038091E1008E7F8093E100A7
:1020E0008091E2008E7F8093E2008091E200806127
:1020F0008093E20042E060E080E00E949A0C8091D0
:10210000F00088608093F0000E948B0AFF91EF91AD
:10211000BF91AF919F918F917F916F915F914F91FF
:102120003F912F910F900FBE0F901F9018951F9207
:102130000F920FB60F9211242F933F934F935F93FB
:102140006F937F938F939F93AF93BF93CF93DF93BF
:10215000EF93FF93C091E900CF708091EC00D82FEE
:10216000D17080FDD0E81092E9008091F000877F67
:102170008093F00078940E94250E1092E9008091DF
:10218000F00088608093F000CD2BCF70C093E90001
:10219000FF91EF91DF91CF91BF91AF919F918F917F
:1021A0007F916F915F914F913F912F910F900FBE53
:1021B0000F901F901895089590936F0280936E0270
:1021C0000895E0916E02F0916F02309721F0019036
:1021D000F081E02D099480E00895EF92FF920F9333
:1021E0001F93CF93DF93E0916E02F0916F023097CF
:1021F000B1F18C010280F381E02D099580914C03AF
:1022000082FF2DC080FF04C08CEA94E00E94EF059D
:10221000E80118E086EAE82E84E0F82E80914C036D
:1022200080FF0BC088811F928F93FF92EF920E94D4
:1022300088060F900F900F900F901150219611115A
:10224000EDCF80914C0380FF0AC084EA94E0DF91D7
:10225000CF911F910F91FF90EF900C94EF05DF91BC
:10226000CF911F910F91FF90EF900895E0916E0232
:10227000F0916F02309721F00480F581E02D0994F0
:102280000895CF93DF9320916C0230916D0228174F
:10229000390709F190936D0280936C02E0916E0210
:1022A000F0916F023097B9F0EC010680F781E02DD4
:1022B000099580914C0382FF0EC080FF0CC0DF9314
:1022C000CF9386E994E09F938F930E9488060F90A6
:1022D0000F900F900F90DF91CF910895CF93DF93E0
:1022E00020916A0230916B022817390709F1909307
:1022F0006B0280936A02E0916E02F0916F02309758
:10230000B9F0EC010084F185E02D099580914C0332
:1023100082FF0EC080FF0CC0DF93CF9386E894E06D
:102320009F938F930E9488060F900F900F900F90AD
:10233000DF91CF9108950C9447120E94F71D0C94E1
:102340001C07BF92CF92DF92EF92FF920F931F93E1
:10235000CF93DF9300D000D01F92CDB7DEB70E949D
:10236000560701E712E0F12C8F2D0E941408B82EB9
:10237000F801C080C82639F4F3940F5F1F4FF0E1D5
:10238000FF12F2CF30C080914C0381FD0E945C129D
:10239000D12CEE24E3948C2D8E21F9F0D982FA828F
:1023A00091E08B2D8E2109F490E09B830E94001E0A
:1023B0008160782F9D838C8349815A816B818D81C7
:1023C0000E94921249815A816B817C818D810E9489
:1023D000781DF80180818E258083D394EE0CF8E07F
:1023E000DF12D9CFC9CF8FEF89838A831B820E94E6
:1023F000001E8160782F9D838C8349815A816B8177
:102400008D810E9492120E94771D0E94C9200E9415
:10241000E11090917002891741F10E94E1108093C0
:10242000700290914C0392FF0EC090FF0CC01F925F
:102430008F9387EB94E09F938F930E9488060F9071
:102440000F900F900F90809170020F900F900F904F
:102450000F900F90DF91CF911F910F91FF90EF9010
:10246000DF90CF90BF900C94891D0F900F900F902C
:102470000F900F90DF91CF911F910F91FF90EF90F0
:10248000DF90CF90BF9008950C941A080895089596
:10249000CF93C62F0E94140821E030E002C0220F23
:1024A000331FCA95E2F790E02823392381E0232BDC
:1024B00009F480E0CF910895EF92FF920F931F935C
:1024C000CF93DF9380ED94E00E94EF05C0E0D0E071
:1024D0008DE2E82E81E0F82E02EC14E08C2F0E94B1
:1024E00014080E94651DFF92EF921F928F93DF9355
:1024F000CF931F930F930E94880621968DB79EB7A6
:1025000008960FB6F8949EBF0FBE8DBFC031D1059F
:1025100029F7DF91CF911F910F91FF90EF900895D0
:1025200008950895CF93DF93CDB7DEB72B970FB6FD
:10253000F894DEBF0FBECDBF942F4F83252F588751
:1025400069877A878B874A855B85452B31F02F3FDA
:1025500031F481E09F3F19F403C081E001C080E0C5
:1025600080FD07C04F81588569857A858B850E94DB
:10257000781DDE01119686E0FD0111928A95E9F73A
:1025800085E0FE01379601900D928A95E1F7498129
:102590005A816B817C818D819E810E94CE192B9600
:1025A0000FB6F894DEBF0FBECDBFDF91CF91089577
:1025B000CF93882309F465C0C82F8CEF8C0F813A24
:1025C00020F080E58C0F8E3248F48C2F0E94F2238D
:1025D000811157C08C2F0E94C21C0CC080E28C0F4E
:1025E000883058F4C77081E001C0880FCA95EAF7B7
:1025F0000E94001DCF910C943A1D8BE58C0F833007
:1026000078F4C53A29F0C63A31F083E890E005C085
:1026100081E890E002C082E890E0CF910C944111F3
:1026200088E58C0F853168F5C83A89F0C93A91F090
:10263000CA3A99F0CB3AA1F0CC3AA9F0CD3AB1F030
:10264000CE3AB9F0CF3AC1F080E090E017C082EE08
:1026500090E014C089EE90E011C08AEE90E00EC0C8
:1026600085EB90E00BC086EB90E008C083EB90E038
:1026700005C084EB90E002C087EB90E0CF910C9412
:102680006E11CF910895882349F19CEF980F913AEC
:1026900020F090E5980F9E3218F40E94DF1C0DC0C8
:1026A00090E2980F983058F4877091E001C0990F2C
:1026B0008A95EAF7892F0E94061D0C943A1D9BE526
:1026C000980F933020F480E090E00C944111885AE8
:1026D000853120F480E090E00C946E1108958823F9
:1026E00021F00E94001D0C943A1D0895882321F0CA
:1026F0000E94061D0C943A1D08950E94201D0E9400
:10270000EF1C0E943A1D0E946F210E943C2080E035
:1027100090E00E94411180E090E00C946E110E94C4
:10272000101D0C947D13CF92DF92EF92FF920F93C6
:102730001F93CF93DF9300D000D01F92CDB7DEB7A9
:102740006C010E948B1D811101C385E0F601DE0141
:10275000119601900D928A95E1F7F6014081518121
:10276000238134812115310531F05F3F31F481E05F
:102770004F3F19F403C081E001C080E080FDE6C254
:10278000F601F280E580E2948FE0E82249835A83E3
:10279000FB82722F3D832C836F2D8D810E94371C0D
:1027A0008C010E94361C0E94261BE12FE295EF70DF
:1027B0008E2F90E0FC01EC5BFF4F0C94AD26812F37
:1027C000807F1F70882311F01295107FFF2049F041
:1027D000112309F452C2812F0E94131D0E943A1D39
:1027E0004CC2802F0E944313112309F4AFC2812FE2
:1027F0000E94191D0F900F900F900F900F90DF9176
:10280000CF911F910F91FF90EF90DF90CF900C949C
:102810003A1D812F807F1F70803211F01295107F3A
:10282000002319F0013009F12BC0FF20A9F0EE20A0
:1028300059F1F1E0812FEF1228C00F900F900F9007
:102840000F900F90DF91CF911F910F91FF90EF901C
:10285000DF90CF900C94231DEE2021F021E0E216B2
:1028600009F474C20E94261D2DC0FF20E9F085E006
:102870008E1508F46BC20E94FD1C812329F022C032
:10288000FF20F1F0E11015C0812F0F900F900F90F5
:102890000F900F90DF91CF911F910F91FF90EF90CC
:1028A000DF90CF900C946F1394E09E1508F44EC205
:1028B00009C0F601858180FFE0C18F708583E4CF78
:1028C000E110EEC1812F61C1812F869586958370BD
:1028D00019F08130B9F03AC2FF2019F0C8019370A5
:1028E00002C080E090E00F900F900F900F900F903B
:1028F000DF91CF911F910F91FF90EF90DF90CF90DC
:102900000C944111FF2019F0C801937002C080E0BF
:1029100090E00F900F900F900F900F90DF91CF915C
:102920001F910F91FF90EF90DF90CF900C946E115C
:10293000802FFF2019F00E944F1F02C00E94B71F76
:102940000F900F900F900F900F90DF91CF911F91EC
:102950000F91FF90EF90DF90CF900C943C20812F4F
:10296000837009F070C0F110F1C1202F22952695D7
:102970002770220F220F602F6F70862F90E0A0E04B
:10298000B0E06C017D01022E04C0CC0CDD1CEE1CFD
:10299000FF1C0A94D2F704FF12C08FE090E0A0E081
:1029A000B0E004C0880F991FAA1FBB1F2A95D2F759
:1029B000BC01CD01609570958095909503C060E055
:1029C00070E0CB011695169513701230B1F040F5FA
:1029D0006C297D298E299F29113031F10F900F909C
:1029E0000F900F900F90DF91CF911F910F91FF905B
:1029F000EF90DF90CF900C944B1B6C297D298E2992
:102A00009F290F900F900F900F900F90DF91CF9113
:102A10001F910F91FF90EF90DF90CF900C94651B6A
:102A20000E944B1BC701B6010F900F900F900F90A3
:102A30000F90DF91CF911F910F91FF90EF90DF905A
:102A4000CF900C94311BFF2019F0812F817001C0B1
:102A50008695882309F47AC1202F22952695277020
:102A6000220F220F602F6F70862F90E0A0E0B0E061
:102A70006C017D01022E04C0CC0CDD1CEE1CFF1C81
:102A80000A94D2F704FF12C08FE090E0A0E0B0E01B
:102A900004C0880F991FAA1FBB1F2A95D2F7BC013B
:102AA000CD01609570958095909503C060E070E0D1
:102AB000CB011695169513701230B1F040F56C29C4
:102AC0007D298E299F29113031F10F900F900F90A1
:102AD0000F900F90DF91CF911F910F91FF90EF908A
:102AE000DF90CF900C94121C6C297D298E299F2990
:102AF0000F900F900F900F900F90DF91CF911F913B
:102B00000F91FF90EF90DF90CF900C94241C0E94C7
:102B1000121CC701B6010F900F900F900F900F90ED
:102B2000DF91CF911F910F91FF90EF90DF90CF90A9
:102B30000C94001C003FC1F128F480E4800F803227
:102B400050F096C0023F09F45EC008F449C0033F4C
:102B500009F46CC08DC0F02FF071EF2E812F8F71B2
:102B6000FF2051F00E94991B802FEE2019F08295D2
:102B7000807F8BCE8F7089CE0E94BA1B802FEE2073
:102B800019F08295807F01C08F700F900F900F9089
:102B90000F900F90DF91CF911F910F91FF90EF90C9
:102BA000DF90CF900C947613FF20A9F024E02E152F
:102BB00008F4CCC0812F8F710F900F900F900F9061
:102BC0000F90DF91CF911F910F91FF90EF90DF90C9
:102BD000CF900C94DF1B85E08E1508F4B7C0EACFC8
:102BE000FF2099F0812F8F710F900F900F900F9011
:102BF0000F90DF91CF911F910F91FF90EF90DF9099
:102C0000CF900C94991BFF2069F3812F8F710F9047
:102C10000F900F900F900F90DF91CF911F910F9118
:102C2000FF90EF90DF90CF900C94BA1BFF2089F0BB
:102C3000812F8F710F900F900F900F900F90DF9159
:102C4000CF911F910F91FF90EF90DF90CF900C9458
:102C5000841B0F900F900F900F900F90DF91CF91EA
:102C60001F910F91FF90EF90DF90CF900C947F1BFE
:102C7000FF2099F0EE2009F4B5CF802F0F900F9030
:102C80000F900F900F90DF91CF911F910F91FF90B8
:102C9000EF90DF90CF900C94D812EE2009F4B5CFCE
:102CA000802F0F900F900F900F900F90DF91CF918A
:102CB0001F910F91FF90EF90DF90CF900C944313F2
:102CC000412F4F70602FC6010E94C51E0F900F90BC
:102CD0000F900F900F90DF91CF911F910F91FF9068
:102CE000EF90DF90CF900C94811A01112FC0FF203C
:102CF00069F10E948F139FEFE0E7F2E09150E0400E
:102D0000F040E1F700C000000F900F900F900F907F
:102D10000F90DF91CF911F910F91FF90EF90DF9077
:102D2000CF900C94671E412F4F70602FC6010F90FB
:102D30000F900F900F900F90DF91CF911F910F91F7
:102D4000FF90EF90DF90CF900C94C81E0F900F90E3
:102D50000F900F900F90DF91CF911F910F91FF90E7
:102D6000EF90DF90CF9008951F93CF93DF9300D023
:102D700000D01F92CDB7DEB7942F4983252F5A83F9
:102D80006B837C838D834C815D81452B31F02F3F9C
:102D900031F481E09F3F19F403C081E001C080E07D
:102DA000182F117080FD31C049815A816B817C815F
:102DB0008D810E94371C292F22952F702C3030F4E2
:102DC0002A30A0F42250223030F022C02C30C9F03A
:102DD0002F30B9F01DC0853A28F48430C0F4823019
:102DE00028F415C090E2980F983088F0883E30F4AF
:102DF000803E68F48450813A58F409C0803F41F421
:102E000006C093FB112710F903C010E001C011E0C8
:102E1000812F0F900F900F900F900F90DF91CF9117
:102E20001F910895CF93DF9300D000D01F92CDB7AC
:102E3000DEB70F900F900F900F900F90DF91CF9112
:102E40000895CF93DF9300D000D000D0CDB7DEB788
:102E500026960FB6F894DEBF0FBECDBFDF91CF919F
:102E60000895CF93DF93C091810280918202C817A9
:102E7000A1F0D0E0CE0166E070E00E948826FC015F
:102E8000ED57FD4F4081518162817381848195812D
:102E90000E9421172196C770E8CFDF91CF91089546
:102EA0004091B3025091B4026091B5027091B602A4
:102EB0008091B7029091B8020C9421171F93CF9381
:102EC000DF938091B80282958F7009F066C080917F
:102ED000B502882309F461C0209181021091820219
:102EE000C091B302D091B402E091B602F091B70262
:102EF00081E0CF3F09F080E0482F211709F44DC051
:102F0000309721F0DF3F21F080E003C081E001C075
:102F1000842F30E080FD3DC0C90166E070E00E9472
:102F20008826DC01AD57BD4F11968C9111978D13FA
:102F300030C08C918C132DC012968C9112978111F8
:102F400028C013968D919C9114978E179F0708F4B3
:102F500001978E1B9F0B883C9105D8F48091B80295
:102F60008F7080618093B802C90166E070E00E94B2
:102F70008826FC01E857FD4F90819F7090619083F7
:102F800083EB92E00E949313DF91CF911F910C94F9
:102F900031172F5F3F4F2770B0CFDF91CF911F9137
:102FA0000895AF92BF92CF92DF92EF92FF920F936C
:102FB0001F93CF93DF93CDB7DEB761970FB6F89429
:102FC000DEBF0FBECDBF7C0185E0F701DE011D969F
:102FD00001900D928A95E1F7D7014C9111962C91B1
:102FE00011971296DC90129713960D911C911497DD
:102FF0005091B3026091B4028091B6029091B702F1
:10300000009731F06F3F31F431E05F3F19F403C0B6
:1030100031E001C030E0B32FB170BB2E30FD76C17E
:10302000A090B502AA2009F4D2C03091B8020817C6
:10303000190728F0F801E81BF90BCF0104C08095AF
:103040009095800F911FCC24C394883C910588F003
:10305000C12C307F09F0A6C0702F198B088B522F1E
:103060006D2D89890E94121783EB92E00E949313C1
:10307000C3C0832F807F09F059C0261315C04513A4
:1030800013C0CD2CD11010C03F7030613093B80206
:103090000E94501783EB92E00E9493138091B80234
:1030A000D70115968C9368C10115110531F02F3F9A
:1030B00031F481E04F3F19F403C081E001C080E0AA
:1030C00080FD03C081E08D2502C080E090E0B82F34
:1030D000B170CB2E80FF1FC0E0918102309182023F
:1030E000E31709F425C1F0E0CF0166E070E00E942B
:1030F0008826DC01AD57BD4F11968C91119728138E
:1031000007C08C91481304C012968C91D81203C04A
:103110003196E770E5CFCD2CDD2009F42DC18091EB
:10312000B80281608093B802C12C26C1261308C062
:10313000451306C0D11004C08091B802D701B9C0B0
:103140004D872E87DF86702F198B088B522F6D2DA0
:1031500089890E94B4168823A1F1DD2091F1209184
:10316000B802822F82958F7090E0029774F0809160
:10317000B3029091B40298878F8319861B870A87C0
:103180002C87CE0107960E94931386E0F701A3EBEC
:10319000B2E001900D928A95E1F70E945E170E94BD
:1031A000501712C0261791F14D872E87DF86702F9A
:1031B000198B088B522F6D2D89890E94B4168111AD
:1031C00039C0C7010E949313CC24C394D5C00817FB
:1031D000190708F447C0F801E81BF90BCF01883C38
:1031E000910508F444C0C12C702F198B088B522F05
:1031F0006D2D89890E941217E3EBF2E086E0DF0172
:103200001D928A95E9F70E945017B6C04513CCCF9E
:10321000D110CACF8091B802F7018583C7010E94FF
:10322000931386E0E3EBF2E0DF011D928A95E9F764
:10323000CA2CA2C0DD2029F22091B802822F8295EB
:103240008F7090E002970CF4A0CF8091B302909120
:10325000B4029A8389831B821D830C832E83CE0143
:10326000019691CF80959095800F911FB8CFCD2C6E
:10327000DD2009F4A6CF261333C0451331C02091B9
:10328000B80220FD24C0822F82958F70482F50E015
:1032900041155105E1F0D70115962C9315974F3044
:1032A000510549F08F5F982F9295907F822F8F70F4
:1032B000892B15968C93C7010E94931386E0F70122
:1032C000A3EBB2E001900D928A95E1F79CCF86E0E6
:1032D000F701A3EBB2E001900D928A95E1F74CC0A3
:1032E0004D872E87DF86702F198B088B522F6D2DFF
:1032F00089890E94B416811148CF8091B8028160FB
:103300008093B802C7010E94931336C0DD2009F4F0
:1033100058CF4D872E87DF86702F198B088B522F41
:103320006D2D89890E94B416882309F44ACF2DCFC8
:10333000702F198B088B522F6D2D89890E94371C95
:10334000292F22952F70223028F49F7039F0811197
:1033500005C00BC0243028F49F7049F4805E88308B
:1033600020F0C7010E949313BC2CCB2C05C0F701A1
:103370009581907F99F7F9CF8C2D61960FB6F894CF
:10338000DEBF0FBECDBFDF91CF911F910F91FF9098
:10339000EF90DF90CF90BF90AF900895CF93DF93E1
:1033A000CDB7DEB72C970FB6F894DEBF0FBECDBFFA
:1033B0004F83588769877A878B879C87CE010796CA
:1033C0000E94D1178823D1F09F8188852A853B856B
:1033D000232B31F08F3F31F481E09F3F19F403C07C
:1033E00081E001C080E080FD6FC04F815885698514
:1033F0007A858B859C850E94211766C086E0FE0138
:103400003796DE01119601900D928A95E1F7FF81C2
:10341000E8856A857B856115710531F0EF3F31F4F0
:1034200081E0FF3F19F403C081E001C080E080FD2E
:103430004BC08091820290E09C012F5F3F4F27702C
:1034400033274091810250E02417350709F443C027
:10345000F983EA837D836C8366E070E00E948826AE
:10346000DC01AD57BD4F96E0FE01319601900D9203
:103470009A95E1F7209382020E94311725C090E0CF
:1034800066E070E00E9488268D579D4F0E94D117FC
:10349000882371F18091810290E066E070E00E94E3
:1034A0008826FC01ED57FD4F408151816281738177
:1034B000848195810E9421178091810290E001967C
:1034C0008770992780938102809181029091820276
:1034D0008913D5CF0DC00E948F13109282021092D3
:1034E0008102E3EBF2E086E0DF011D928A95E9F7C5
:1034F0002C960FB6F894DEBF0FBECDBFDF91CF91F3
:103500000895DF92EF92FF920F931F93CF93DF9373
:10351000FC01892B09F488C0E12CF12CDD24D39423
:10352000EF0121968491853709F460C058F48437FF
:1035300008F04EC0843008F068C08130D1F082308D
:1035400071F172C0883709F45BC050F4863709F412
:1035500053C0873709F068C08E2D0E940D1D52C0E0
:103560009CE7980F903708F05FC08F770E94431355
:103570004EC08F010E5F1F4FFE01849190E2980FA5
:10358000983050F48770FD2D01C0FF0F8A95EAF73F
:103590008F2F0E94131D15C00E94D81214C08F01D6
:1035A0000E5F1F4FFE01849190E2980F983068F4EF
:1035B0008770FD2D01C0FF0F8A95EAF78F2F0E94BB
:1035C000191D0E943A1DE80122C00E944313FBCF3F
:1035D000CF010296FE01C491CC2361F0EFE9FFE038
:1035E0003197F1F700C00000C150F6CFCF0102962D
:1035F000FE01F490EC010BC00E94FD1CE82E07C0F8
:103600000E94101D0E943A1D02C00E94D8128F2DE8
:10361000882341F0EFE9FFE03197F1F700C00000A7
:103620008150F6CFFE017CCFDF91CF911F910F919A
:10363000FF90EF90DF9008956093390370933A0301
:1036400080933B0390933C030C94881D08956093F2
:103650003D0370933E0380933F03909340030C948B
:10366000871D0F931F9300913D0310913E032091FE
:103670003F0330914003602B712B822B932B60937F
:103680003D0370933E0380933F03909340031F914B
:103690000F910C94871D0F931F9300913D03109180
:1036A0003E0320913F033091400360237123822326
:1036B000932360933D0370933E0380933F03909365
:1036C00040031F910F910C94871D0F931F9300913E
:1036D0003D0310913E0320913F033091400360274A
:1036E00071278227932760933D0370933E03809355
:1036F0003F03909340031F910F910C94871D60E04E
:1037000070E0CB010C941C1B0F931F9341E050E021
:1037100060E070E08A019B0104C0000F111F221FAE
:10372000331F8A95D2F7C901B8011F910F910C94EC
:103730001C1B0F931F9341E050E060E070E004C059
:10374000440F551F661F771F8A95D2F78091390362
:1037500090913A03A0913B03B0913C038A019B01F5
:10376000082B192B2A2B3B2BC901B8011F910F9154
:103770000C941C1B0F931F9341E050E060E070E03D
:1037800004C0440F551F661F771F8A95D2F74095D6
:103790005095609570958091390390913A03A0916E
:1037A0003B03B0913C038A019B01082319232A2380
:1037B0003B23C901B8011F910F910C941C1B0F935F
:1037C0001F9341E050E060E070E004C0440F551FDB
:1037D000661F771F8A95D2F78091390390913A033B
:1037E000A0913B03B0913C038A019B010827192754
:1037F0002A273B27C901B8011F910F910C941C1B6C
:103800000F931F930091390310913A0320913B03CA
:1038100030913C03602B712B822B932B1F910F91C6
:103820000C941C1B0F931F930091390310913A03C2
:1038300020913B0330913C03602371238223932327
:103840001F910F910C941C1B0F931F930091390330
:1038500010913A0320913B0330913C03602771277C
:10386000822793271F910F910C941C1B08958F9210
:103870009F92AF92BF92DF92EF92FF920F931F93AE
:10388000CF93DF9300D000D01F92CDB7DEB76B830C
:103890007C838D838A018C819D81892B31F01F3F30
:1038A00031F481E04F3F19F403C081E001C080E0B2
:1038B00080FF03C080E090E054C08B81882309F42E
:1038C0003DC08090390390903A03A0903B03B090A4
:1038D0003C0380913D0390913E03A0913F03B09142
:1038E0004003882A992AAA2ABB2A2FE1E22EF12C2A
:1038F000D501C4010E2C04C0B695A7959795879560
:103900000A94D2F780FD06C081E0E81AF10880F73A
:10391000D12C07C0DE2CB8018E2D0E94981E019775
:1039200099F3E12FF0E093E0EE0FFF1F9A95E1F796
:10393000E754FD4FE00FF11DD0820CC0E12FF0E005
:1039400083E0EE0FFF1F8A95E1F7E754FD4FE00F8C
:10395000F11DD08009831A8369817A818D2D0E949F
:10396000981E0F900F900F900F900F90DF91CF91B6
:103970001F910F91FF90EF90DF90BF90AF909F90BD
:103980008F9008952091110130911201F901329622
:103990009FEF40E05191851789F09F3F19F4511135
:1039A00001C0942F4F5F4630A9F79F3F39F0F901CE
:1039B000E90FF11D97FDFA95828308950895E0912E
:1039C0001101F09112019F012A5F3F4F92818913EB
:1039D00001C012823196E217F307C1F7089581E022
:1039E00090E0E0911101F0911201E80FF91F1082AF
:1039F000019688309105A9F7089580914B030895A9
:103A000090914B03892B80934B030895809590915F
:103A10004B03892380934B03089580934B030895B0
:103A200010924B03089590914A03892B80934A0387
:103A30000895809590914A03892380934A030895BD
:103A400010924A0308958093410308951092410310
:103A500008958091110190911201FC0131969C0111
:103A6000285F3F4F80E0919191118F5FE217F3073C
:103A7000D1F70895E0911101F091120180914B036B
:103A80008083E0911101F0911201908180914A03AD
:103A9000892B808380914103882361F0E09111019B
:103AA000F09112019081892B80830E94291D811140
:103AB0001092410380911101909112010C94ED102C
:103AC00090933F0180933E0108958295982F9373C0
:103AD000292F220F220F982F9C7C96959695922B3A
:103AE000892F8575880F9A7A9695892B0895089560
:103AF000CF93DF9300D000D01F92CDB7DEB70F90E9
:103B00000F900F900F900F90DF91CF91089508952F
:103B100008950C94441280E00895809161038430EC
:103B200021F110924D0320E488E190E00FB6F89463
:103B3000A895809360000FBE2093600083B7817FBB
:103B4000846083BF83B7816083BF7894889583B78F
:103B50008E7F83BF0FB6F894A8958091600088612E
:103B600080936000109260000FBE0895CF930E9472
:103B700090120E9456070E949112C0E08C2F0E9462
:103B80001408811104C0CF5FC031C1F701C081E0CA
:103B9000CF9108950E9446120C948F131F920F929A
:103BA0000FB60F9211248F939F93AF93BF93809181
:103BB0004D03811113C080914E0390914F03A0914A
:103BC0005003B09151034196A11DB11D80934E0346
:103BD00090934F03A0935003B0935103BF91AF91C3
:103BE0009F918F910F900FBE0F901F90189582E0BC
:103BF00084BD93E095BD9AEF97BD80936E000895C4
:103C00002FB7F89480914E0390914F03A0915003E9
:103C1000B09151032FBF08952FB7F89460914E03D0
:103C200070914F0380915003909151032FBF0895DD
:103C3000CF92DF92EF92FF920F931F932FB7F894DA
:103C400040914E0350914F03609150037091510386
:103C50002FBF6A017B01EE24FF248C0120E030E0BD
:103C6000C016D106E206F30610F4415051099A013C
:103C7000281B390BC9011F910F91FF90EF90DF9026
:103C8000CF9008951F920F920FB60F9211248F9329
:103C90009F93AF93BF9380914E0390914F03A09158
:103CA0005003B09151030196A11DB11D80934E03A5
:103CB00090934F03A0935003B0935103BF91AF91E2
:103CC0009F918F910F900FBE0F901F9018950E949B
:103CD000850FF89487E797E7909301088093000891
:103CE00087E090EBDC0180936A0390936B03A093D1
:103CF0006C03B0936D039CE088E10FB6F894A8952F
:103D0000809360000FBE90936000FFCFE92FF0E03A
:103D100093E0EE0FFF1F9A95E1F7E80FF11DE855CC
:103D2000FF4F8491982F92959F708F709770089590
:103D3000CF93C82FCB010E94861E292F30E054E07C
:103D4000220F331F5A95E1F7282B203831051CF03C
:103D500080E090E018C0EC2FF0E023E0EE0FFF1FB2
:103D60002A95E1F79770E90FF11D34E0EE0FFF1F80
:103D70003A95E1F78F70E80FF11DEE0FFF1FE0504D
:103D8000F84985919491CF91089580E090E008954D
:103D900008958091540380FF0CC08091160190E03B
:103DA00065E070E00E9488269595879595958795A2
:103DB0002EC081FF0AC08091160190E065E070E09E
:103DC0000E9488269595879522C082FF08C0809121
:103DD000160190E065E070E00E94882618C02091EE
:103DE00055032223D9F030911501231780F78091D4
:103DF000160190E065E070E00E948826622F70E076
:103E00000E948826632F70E00E949926CB0180389B
:103E1000910538F4009739F481E005C085E090E021
:103E200008958FE7089508958091540380FF08C096
:103E30006091140170E0759567957595679523C03D
:103E400081FF06C06091140170E0759567951BC0F5
:103E500082FF04C06091140170E012C060915503AC
:103E60006623A9F0209113016217A0F78091140135
:103E700070E090E00E948826622F70E00E949926F0
:103E80006038710540F46115710519F406C061E0F0
:103E900070E0862F08958FE7089581E00895803FB0
:103EA00021F40E94C91E819504C0813F29F40E941B
:103EB000C91E809358030895823F21F40E94C91EB1
:103EC000819504C0833F29F40E94C91E8093570343
:103ED0000895893F19F40E94141F05C08A3F31F4E8
:103EE0000E94141F81958093590308958B3F21F4FC
:103EF0000E94141F819504C08C3F29F40E94141F56
:103F000080935A030895843F21F480915603816081
:103F100017C0853F21F480915603826011C0863F0F
:103F200021F48091560384600BC0873F21F4809177
:103F30005603886005C0883F31F480915603806144
:103F40008093560308958D3F21F48091540381603E
:103F50000BC08E3F21F480915403826005C08F3FD7
:103F600029F4809154038460809354030895803F22
:103F700039F48091580387FF6CC01092580369C0D0
:103F8000813F29F4809158031816BCF362C09091C8
:103F90005703823F29F497FF5CC01092570359C022
:103FA000833F19F41916CCF354C0893F41F4809132
:103FB000590318160CF04DC0109259034AC08A3F9D
:103FC00029F48091590387FF44C0F6CF8B3F39F421
:103FD00080915A0387FF3DC010925A033AC08C3F2C
:103FE00029F480915A031816BCF333C0843F21F49E
:103FF000809156038E7F17C0853F21F48091560330
:104000008D7F11C0863F21F4809156038B7F0BC0BA
:10401000873F21F480915603877F05C0883F31F4A4
:10402000809156038F7E8093560313C08D3F21F4F9
:10403000809154038E7F0BC08E3F21F480915403F6
:104040008D7F05C08F3F29F4809154038B7F80932F
:1040500054038091570381110EC080915803811140
:104060000AC080915903811106C080915A038111C1
:1040700002C010925503089580914C0383FF7EC0C7
:1040800085E095E00E94EF05809156031F928F9383
:1040900080E095E09F938F930E9488068EEF94E0D6
:1040A0000E94EF0580915703282F082E000C330B38
:1040B0003F938F938BEF94E09F938F930E9488069A
:1040C00089EF94E00E94EF0580915803282F082E75
:1040D000000C330B3F938F9386EF94E09F938F9365
:1040E0000E94880684EF94E00E94EF0580915903B6
:1040F000282F082E000C330B3F938F9381EF94E011
:104100009F938F930E9488068FEE94E00E94EF05A4
:1041100080915A03282F082E000C330B3F938F9366
:104120008CEE94E09F938F930E94880689EE94E032
:104130000E94EF05809155031F928F9386EE94E0C5
:104140009F938F930E94880684EE94E00E94EF056F
:10415000809154031F928F9381EE94E09F938F93ED
:104160000E9488068EED94E00E94EF058DB79EB701
:104170004C960FB6F8949EBF0FBE8DBF86E593E0B8
:104180000E9436110E94001E9093530380935203A5
:1041900008951F93CF93DF9380915203909153031F
:1041A0000E94181EFC0120915503222321F08091CA
:1041B000170190E007C08091180190E06AE070E07C
:1041C0000E948826E817F90708F485C080915703F4
:1041D000C0915803D091590310915A03811107C01F
:1041E000C11175C0D11173C0111171C074C02F3FBE
:1041F00019F02F5F20935503181624F40E94C91E4E
:10420000809357038091570387FF05C00E94C91E02
:104210008195809357031C1624F40E94C91E809335
:1042200058038091580387FF05C00E94C91E8195DD
:104230008093580360915703662331F1C09158036E
:10424000CC2311F1062E000C770B880B990B0E94E2
:10425000872523E333E343E35FE30E94EB250E94DA
:104260004F25609357036C2FCC0F770B880B990B5E
:104270000E94872523E333E343E35FE30E94EB25BA
:104280000E944F25609358031D1624F40E94141FAA
:10429000809359038091590387FF05C00E94141F22
:1042A000819580935903111624F40E94141F809362
:1042B0005A0380915A0387FF05C00E94141F8195FD
:1042C00080935A03DF91CF911F910C943C202F3F94
:1042D00009F08FCFA0CFDF91CF911F910895E6E530
:1042E000F3E085E0DF011D928A95E9F7109255030E
:1042F00010925403089588E297E00E94EF051F9200
:1043000081E08F931F9285E08F938AED96E09F93D3
:104310008F930E9488060F900F900F900F900F9030
:104320000F9008958330E9F128F4813061F08230F4
:1043300009F10895853009F462C008F449C0863057
:1043400009F474C0089580911801262F30E0280FD9
:10435000311D2F3F310524F4680F6093180103C00D
:104360008FEF80931801809118011F928F9383E142
:1043700096E072C080911701262F30E0280F311D82
:104380002F3F310524F4680F6093170103C08FEFAE
:1043900080931701809117011F928F9381E096E01F
:1043A0005BC080911601262F30E0280F311D2F3F72
:1043B000310524F4680F6093160103C08FEF8093DA
:1043C0001601809116011F928F938EEE95E044C0E6
:1043D00080911501262F30E0280F311D2F3F310528
:1043E00024F4680F6093150103C08FEF80931501CB
:1043F000809115011F928F9389ED95E02DC08091DA
:104400001401262F30E0280F311D2F3F310524F4F1
:10441000680F6093140103C08FEF809314018091A3
:1044200014011F928F9380EC95E016C080911301C8
:10443000262F30E0280F311D2F3F310524F4680F5F
:104440006093130103C08FEF8093130180911301D8
:104450001F928F9385EA95E09F938F930E94880621
:104460000F900F900F900F900895833081F128F4F2
:10447000813059F08230D1F00895853009F449C077
:10448000B8F1863009F456C0089580911801681774
:1044900020F4861B8093180102C0109218018091AD
:1044A00018011F928F9386E995E054C080911701FF
:1044B000681720F4861B8093170102C01092170121
:1044C000809117011F928F9384E895E043C08091FB
:1044D0001601681720F4861B8093160102C0109203
:1044E0001601809116011F928F9381E795E032C0EB
:1044F00080911501681720F4861B8093150102C076
:1045000010921501809115011F928F938CE595E013
:1045100021C080911401681720F4861B8093140138
:1045200002C010921401809114011F928F9383E4B2
:1045300095E010C080911301681720F4861B8093CA
:10454000130102C010921301809113011F928F93E7
:1045500088E295E09F938F930E9488060F900F90BA
:104560000F900F900895CF93C82F1F928F938DE2D5
:1045700098E09F938F930E94880681E090E0A0E0EE
:10458000B0E0BC01CD0104C0660F771F881F991FE2
:10459000CA95D2F70E94271B0F900F900F900F9093
:1045A000CF910C948F13CF93873288F58E3108F01A
:1045B0000BC18E3009F487C0D8F4873009F460C08D
:1045C0008B3009F44FC0863009F002C180914C0352
:1045D000817F8E7F80934C0382E398E00E94EF05F9
:1045E0008BEF9AE00E94EF0581E080935C0346C068
:1045F000863109F4B0C020F4803109F47AC0E8C0F3
:10460000893109F491C08B3109F449C0E1C0883384
:1046100049F150F4893209F4D5C0853309F4D2C088
:10462000873209F0D5C0CEC0833409F4CBC028F45A
:104630008A3308F4CDC08953C8C0883409F0C8C093
:104640000E948F138AEE9AE00E94EF052FEF83ED10
:1046500090E3215080409040E1F700C000000E94AC
:10466000671E0CC089E598E041C081ED9AE00E9488
:10467000EF0580914C03816080934C03C1E0ADC095
:1046800080914C03C82FC17080FFEFCF8DED9AE071
:104690000E94EF0580914C03817F8E7F3FC09091F7
:1046A0004C0391FBCC27C0F981E0C827892FC0FBC0
:1046B00081F980934C03CC2319F084EC9AE029C053
:1046C00086EB9AE013C090914C0392FBCC27C0F983
:1046D00081E0C827892FC0FB82F980934C03CC234B
:1046E00019F087EA9AE015C087E99AE00E94EF0581
:1046F000C5CF90914C0393FBCC27C0F981E0C8272C
:10470000892FC0FB83F980934C03CC2351F08BE8B5
:104710009AE00E94EF0580914C03816080934C03E6
:104720005CC08EE79AE0E2CF8FE69AE00E94EF0548
:1047300080E49AE00E94EF058BEF99E00E94EF057C
:1047400083ED99E00E94EF0583E899E00E94EF0570
:1047500087E599E0CBCF89E499E00E94EF050E94BC
:10476000E1101F928F938FE299E09F938F930E94A5
:104770008806809110011F928F9388E199E09F93A2
:104780008F930E948806809169021F928F9385E023
:1047900099E09F938F930E9488060E940C1E9F931E
:1047A0008F937F936F938EEE98E09F938F930E94E9
:1047B00088068DB79EB742960FB6F8949EBF0FBE7F
:1047C0008DBF5CCF80E001C08D510E94B32256CFD7
:1047D0008CEE98E00E94EF05C0E08C2FCF910895F9
:1047E00080E00895CF93C82F80915C03813091F0D1
:1047F00020F0823009F453C04AC1E0911101F091D8
:1048000012018081843489F0883879F0823209F08D
:1048100040C10BC0E0911101F091120180818434FC
:1048200021F0883811F0823261F48C2F0E94360812
:10483000811104C08C2F0E94D3222FC081E090E010
:104840002CC08C2F0E94F023811126C0C431E1F0CE
:1048500070F4CB3081F0C031D1F40E947B2185E22D
:1048600098E00E94EF0582E080935C0315C0C93296
:1048700059F0C83361F482E398E00E94EF0589E2C1
:1048800098E00E94EF0508C010925C0304C183E227
:1048900098E00E94EF05FFC081E08170FEC0C43245
:1048A00028F5CE3108F0C1C0CB30A1F1D0F4C7302B
:1048B00009F0D3C08EE18093180182E38093170141
:1048C0008AE08093160184E18093150188E080934B
:1048D000140188E28093130189EC96E00E94EF05B1
:1048E000BFC0C33149F1C431C1F0B7C0CB3409F402
:1048F000A9C028F4C93289F0C83361F0AEC0C1350F
:1049000009F49EC0C23509F499C0CE3409F0A5C09F
:104910006AE09EC00E947B21A3C080915B03882334
:1049200019F010925B039CC086ED96E00E94EF05A3
:1049300081E080935C03B1C080EB96E00E94EF05BC
:104940008EE996E00E94EF05809118011F928F93E7
:104950008BE996E09F938F930E94880689E996E001
:104960000E94EF0587E896E00E94EF05809117010D
:104970001F928F9384E896E09F938F930E948806FE
:1049800082E896E00E94EF0583E796E00E94EF053B
:10499000809116011F928F9380E796E09F938F93EB
:1049A0000E9488068EE696E00E94EF058DE596E06F
:1049B0000E94EF05809115011F928F938AE596E082
:1049C0009F938F930E94880688E596E00E94EF05EA
:1049D00083E496E00E94EF05809114011F928F936B
:1049E00080E496E09F938F930E9488068EE396E082
:1049F0000E94EF0587E296E00E94EF058091130187
:104A00001F928F9384E296E09F938F930E94880673
:104A100082E296E00E94EF058DB79EB748960FB6EA
:104A2000F8949EBF0FBE8DBF1BC0CE51EC2FF0E09F
:104A3000EC5CFE4F808180935B0312C061E003C099
:104A400061E006C06AE080915B030E94922108C089
:104A500080915B030E94352203C087EC96E013C06F
:104A600080915B03882369F01F928F9381EC96E01D
:104A70009F938F930E9488060F900F900F900F9036
:104A800004C08EEB96E00E94EF0581E006C0109214
:104A90005C0380E002C080E000CFCF9108950E94C7
:104AA00056256894B1110C94E52508950E94CA25F5
:104AB00088F09F5798F0B92F9927B751B0F0E1F0DF
:104AC000660F771F881F991F1AF0BA95C9F714C08F
:104AD000B13091F00E94E425B1E008950C94E425F2
:104AE000672F782F8827B85F39F0B93FCCF38695C8
:104AF00077956795B395D9F73EF490958095709525
:104B000061957F4F8F4F9F4F0895E89409C097FBA1
:104B10003EF490958095709561957F4F8F4F9F4F94
:104B20009923A9F0F92F96E9BB279395F6958795D8
:104B300077956795B795F111F8CFFAF4BB0F11F49B
:104B400060FF1BC06F5F7F4F8F4F9F4F16C0882342
:104B500011F096E911C0772321F09EE8872F762F78
:104B600005C0662371F096E8862F70E060E02AF0B9
:104B70009A95660F771F881FDAF7880F96958795A5
:104B800097F9089557FD9058440F551F59F05F3F0E
:104B900071F04795880F97FB991F61F09F3F79F05F
:104BA00087950895121613061406551FF2CF4695E1
:104BB000F1DF08C0161617061806991FF1CF869563
:104BC0007105610508940895E894BB276627772747
:104BD000CB0197F908950E94FD250C9477260E9439
:104BE000692638F00E94702620F0952311F00C946D
:104BF00060260C9466260C94E5250E94C22578F365
:104C00009923C9F35523B9F3950F50E0551FAA27EF
:104C1000EE27FF27BB2700240894679520F4E20FB6
:104C2000F31FB41F0A1E220F331F441FAA1F6695CD
:104C3000A9F7779530F4F30FB41F0A1E121E08F47B
:104C40006395330F441FAA1F221F769599F7879506
:104C500020F4B40F0A1E121E631F440FAA1F221F46
:104C6000331F8695A9F7862F712D602D11249F572C
:104C700050409AF0F1F088234AF0EE0FFF1FBB1F5F
:104C8000661F771F881F91505040A9F79E3F51051E
:104C900080F00C9460260C94E5255F3FE4F3983E89
:104CA000D4F3869577956795B795F795E7959F5FC8
:104CB000C1F7FE2B880F911D9695879597F908955A
:104CC00097F99F6780E870E060E008959FEF80ECBF
:104CD000089500240A941616170618060906089562
:104CE00000240A9412161306140605060895092EC8
:104CF0000394000C11F4882352F0BB0F40F4BF2B37
:104D000011F460FF04C06F5F7F4F8F4F9F4F089576
:104D10000024552704C0080E591F880F991F0097BB
:104D200029F076956795B8F37105B9F7802D952F21
:104D3000089597FB072E16F4009407D077FD09D04D
:104D40000E94B32607FC05D03EF4909581959F4FB5
:104D50000895709561957F4F0895EE0FFF1F0590A0
:104D6000F491E02D0994AA1BBB1B51E107C0AA1FB7
:104D7000BB1FA617B70710F0A61BB70B881F991FFC
:104D80005A95A9F780959095BC01CD010895F894A6
:024D9000FFCF53
:104D92000560010000FFC60856093309FD08C9086D
:104DA2000142032808140A321E404D36224604F9F5
:104DB20003C303A1032D0346035F03780300000826
:0E4DC2000004000201020304050607080900B0
:106800008800EA44E944E244040005000600070069
:10681000080009000A000B000C000D000E000F001C
:1068200010001100120013001400150016001700CC
:10683000180019001A001B001C001D001E001F007C
:10684000200021002200230024002500260027002C
:10685000280029002A002B002C002D002E002F00DC
:1068600030003100000033003400350036003700BE
:10687000380039003A003B003C003D003E003F003C
:1068800040004100420043004400450046004700EC
:10689000480049004A004B004C004D004E004F009C
:1068A000500051005200530054005500560057004C
:1068B000580059005A005B005C005D005E005F00FC
:1068C0006000610062006300640065A100000000D8
:1068D000680069006A006B006C006D006E006F005C
:1068E0007000710072007300000087008A008B0046
:1068F000E000E100E200E3008140E500E600E7009F
:106900000100010001000100EA4401000100E2442D
:106910000100010001000100460001004A004B0097
:10692000010001004700480001000100E9440100A6
:106930000100010001000100010001003A003B00DC
:106940003C003D003E003F0040004100420043004B
:106950000100350001000100010044004500520023
:1069600001004900000050004F004C004D004E0057
:1069700051000100010001000100010001000100BF
:1069800001000100010001000100010001000100FF
:1069900001000100010001000100010001000100EF
:1069A00001000100010001000100010001000100DF
:1069B00001000100010001000100010001000100CF
:1069C00001000100010001000100010000000000C1
:1069D00001000100010001000100010001000100AF
:1069E00001000100010001000000010001000100A0
:1069F000010001000100010000E0010001000100B0
:00000001FF
